:06080000C2857F327E007C
:10080600E4FDFCC3ED9FEC9E5015E4FBFA0BBB0028
:0F081600010ABA04F8BBFBF50DBD00010C80E42C
:0108250022B0
:09087D00D281C282D283C285221D
:10084900C281C282D283120800C281C282C283C21B
:040859008502080606
:10085D00D281C282C283120800C281C282C283C207
:04086D0085020806F2
:10082600D290D294D280D2842090083094051208B7
:100836005D80F530900820940512084980EA120878
:030846007D80E5CD
:0300000002087182
:0C087100787FE4F6D8FD758107020826A8
:00000001FF
